:020000020000FC
:1000000012C01895189518951895189541C042C0BA
:100010001895189518951895189518951895189578
:100020001895189518950FE50DBF04E00EBF0FEF5A
:1000300004BB00E001BB0FEF05BB80E29EE49BBD6B
:100040008ABD8CED95E099BD88BD09B7086109BFEF
:100050000AE00EBD789487990CC088B599B508E080
:10006000091719F40CEF081721F0019699BD88BD06
:1000700013D086990CC088B599B502E0091719F418
:100080000CEB081721F0019799BD88BD05D0E3CF8F
:10009000A99A1895A99818950FEF00000000000084
:0600A0000A95D9F708954E
:00000001FF
